Fix another crash in the recover extension triggered by a corrupt database.

FossilOrigin-Name: d125377378916fb3147612a536fde15ee955176eea9ea6eaa4a2ee5f1e8e1cbe
This commit is contained in:
dan 2022-10-27 20:27:45 +00:00
parent 10f5525410
commit 676d1cda92
5 changed files with 139 additions and 13 deletions

View File

@ -103,8 +103,8 @@ struct DbdataCursor {
/* Only for the sqlite_dbdata table */
u8 *pRec; /* Buffer containing current record */
int nRec; /* Size of pRec[] in bytes */
int nHdr; /* Size of header in bytes */
sqlite3_int64 nRec; /* Size of pRec[] in bytes */
sqlite3_int64 nHdr; /* Size of header in bytes */
int iField; /* Current field number */
u8 *pHdrPtr;
u8 *pPtr;
@ -639,6 +639,7 @@ static int dbdataNext(sqlite3_vtab_cursor *pCursor){
}
iHdr = dbdataGetVarintU32(pCsr->pRec, &nHdr);
if( nHdr>nPayload ) nHdr = 0;
pCsr->nHdr = nHdr;
pCsr->pHdrPtr = &pCsr->pRec[iHdr];
pCsr->pPtr = &pCsr->pRec[pCsr->nHdr];

View File

@ -156,7 +156,6 @@ do_test 4.0 {
| 16: 00 01 01 02 00 40 20 20 01 00 ff 00 42 01 10 01 .....@ ....B...
| 32: ef 00 00 87 00 ff ff ff f0 01 01 10 ff ff 00 00 ................
| end crash-00f2d3627f1b43.db
.recover
}]} {}
do_test 4.1 {
@ -165,5 +164,131 @@ do_test 4.1 {
list [catch { $R finish } msg] $msg
} {1 {unable to open database file}}
#-------------------------------------------------------------------------
#
reset_db
do_test 5.0 {
sqlite3 db {}
db deserialize [decode_hexdb {
.open --hexdb
| size 16384 pagesize 4096 filename crash-7b75760a4c5f15.db
| page 1 offset 0
| 0: 53 51 4c 69 74 65 20 66 6f 72 6d 61 74 20 33 00 SQLite format 3.
| 16: 10 00 01 01 00 40 20 20 00 00 00 00 00 00 00 04 .....@ ........
| 32: 00 00 00 00 00 00 00 00 00 00 00 03 00 00 00 00 ................
| 96: 00 00 00 00 0d 00 00 00 03 0f 4e 00 0f bc 0f 90 ..........N.....
| 112: 0f 4e 00 00 00 00 00 00 00 00 00 00 00 00 00 00 .N..............
| 3904: 00 00 00 00 00 00 00 00 00 00 00 00 00 00 40 03 ..............@.
| 3920: 06 17 11 11 01 6d 74 61 62 6c 65 74 32 74 32 04 .....mtablet2t2.
| 3936: 43 52 45 41 54 45 20 54 41 42 4c 45 20 74 32 28 CREATE TABLE t2(
| 3952: 78 2c 79 2c 7a 20 50 52 49 4d 41 52 59 20 4b 45 x,y,z PRIMARY KE
| 3968: 59 29 20 57 49 54 48 4f 55 54 20 52 4f 57 49 44 Y) WITHOUT ROWID
| 3984: 2a 02 06 17 13 11 01 3f 69 6e 64 65 78 74 31 61 *......?indext1a
| 4000: 74 31 03 43 52 45 41 54 45 20 49 4e 44 45 58 20 t1.CREATE INDEX
| 4016: 74 31 61 20 4f 4e 20 74 31 28 61 29 42 01 06 17 t1a ON t1(a)B...
| 4032: 11 11 01 71 74 61 62 6c 65 74 31 74 31 02 43 52 ...qtablet1t1.CR
| 4048: 45 41 54 45 20 54 41 42 4c 45 20 74 31 28 61 20 EATE TABLE t1(a
| 4064: 49 4e 54 2c 62 20 54 45 58 54 2c 63 20 42 4c 4f INT,b TEXT,c BLO
| 4080: 42 2c 64 20 52 45 41 4c 29 20 53 54 52 49 43 54 B,d REAL) STRICT
| page 2 offset 4096
| 0: 0d 00 00 00 14 0c ae 00 0f df 0f bd 0f 9a 0f 76 ...............v
| 16: 0f 51 0f 2b 0f 04 0e dc 0e b3 0e 89 0e 5e 0e 32 .Q.+.........^.2
| 32: 0e 05 0d 1a 0d a8 0d 78 0d 47 0d 15 0c e2 00 00 .......x.G......
| 3232: 00 00 00 00 00 00 00 00 00 00 00 00 00 00 32 14 ..............2.
| 3248: 05 06 3f 34 07 15 f4 c9 23 af e2 b3 b6 61 62 63 ..?4....#....abc
| 3264: 30 32 30 78 79 7a 01 00 00 00 00 00 00 00 00 00 020xyz..........
| 3280: 00 00 00 00 00 00 00 00 00 00 c3 b0 96 7e fb 4e .............~.N
| 3296: c5 4c 31 13 05 06 1f 32 07 dd f2 2a a5 7e b2 4d .L1....2...*.~.M
| 3312: 82 61 62 63 30 31 39 78 79 7a 01 00 00 00 00 00 .abc019xyz......
| 3328: 00 00 00 00 00 00 00 00 00 00 00 00 00 c3 a3 d6 ................
| 3344: e9 f1 c2 fd f3 30 12 05 06 1f 30 07 8f 8f f5 c4 .....0....0.....
| 3360: 35 b6 7f 8d 61 62 63 30 31 38 00 00 00 00 00 00 5...abc018......
| 3376: 00 00 00 00 00 00 00 00 00 00 00 00 00 00 00 43 ...............C
| 3392: b2 13 1f 9d 56 8a 47 21 b1 05 06 1f 2e 07 7f 46 ....V.G!.......F
| 3408: 91 03 3f 97 fb f7 61 62 63 30 00 00 00 00 00 00 ..?...abc0......
| 3440: c3 bb d8 96 86 c2 e8 2b 2e 10 05 06 1f 2c 07 6d .......+.....,.m
| 3456: 85 7b ce d0 32 d2 54 61 62 63 30 00 00 00 00 00 ....2.Tabc0.....
| 3488: 43 a1 eb 44 14 dc 03 7b 2d 0f 05 06 1f 2a 07 d9 C..D....-....*..
| 3504: ab ec bf 34 51 70 f3 61 62 63 30 31 35 78 79 7a ...4Qp.abc015xyz
| 3520: 00 00 00 00 00 00 00 00 00 00 00 00 00 00 00 c3 ................
| 3536: b6 3d f4 46 b1 6a af 2c 0e 05 06 1f 28 07 36 75 .=.F.j.,....(.6u
| 3552: e9 a2 bd 05 04 ea 61 62 63 30 31 34 78 79 7a 00 ......abc014xyz.
| 3568: 00 00 00 00 00 00 00 00 00 00 00 00 00 c3 ab 23 ...............#
| 3584: a7 6a 34 ca f8 2b 0d 05 06 1f 26 07 48 45 ab e0 .j4..+....&.HE..
| 3600: 8c 7c ff 0c 61 62 63 30 31 33 78 79 7a 00 00 00 .|..abc013xyz...
| 3616: 00 00 00 00 0d d0 00 00 00 00 43 b8 d3 93 f4 92 ..........C.....
| 3632: 5b 7a 2a 0c 05 06 1f 24 07 be 6d 1e db 61 5d 80 [z*....$..m..a].
| 3648: 9f 61 62 63 30 31 32 78 79 7a 00 00 00 00 00 00 .abc012xyz......
| 3664: 00 00 00 00 00 00 43 b5 a1 a4 af 7b c6 60 29 0b ......C......`).
| 3680: 05 06 1f 22 07 6e a2 a3 64 68 d4 a6 bd 61 62 63 .....n..dh...abc
| 3696: 30 31 31 78 79 7a 00 00 00 00 00 00 00 00 00 00 011xyz..........
| 3712: 00 c3 c4 1e ff 0f fc e6 ff 28 0a 05 06 1f 20 07 .........(.... .
| 3728: 50 f9 4a bb a5 7a 1e ca 61 62 63 30 31 30 78 79 P.J..z..abc010xy
| 3744: 7a 00 00 00 00 00 00 00 00 00 00 c3 a7 90 ed d9 z...............
| 3760: 5c 2c d5 27 09 05 06 1f 1e 07 90 8e 1d d9 1c 3a .,.'...........:
| 3776: e8 c1 61 62 63 30 30 39 78 79 7a 00 00 00 00 00 ..abc009xyz.....
| 3792: 00 00 00 00 43 a7 97 87 cf b0 ff 79 26 08 05 06 ....C......y&...
| 3808: 1f 1c 07 86 65 f6 7c 50 7a 2c 76 61 62 63 30 30 ....e.|Pz,vabc00
| 3824: 38 78 79 7a 00 00 00 00 00 00 00 00 c3 b0 e3 4c 8xyz...........L
| 3840: 4f d3 41 b5 25 07 05 06 1f 1a 07 8b 20 e5 68 11 O.A.%....... .h.
| 3856: 13 55 87 61 62 63 30 30 37 78 79 7a 00 00 00 00 .U.abc007xyz....
| 3872: 00 00 00 c3 b6 a3 74 f1 9c 33 f8 24 06 05 06 1f ......t..3.$....
| 3888: 18 07 97 3c bc 34 49 94 54 ab 61 62 63 30 30 36 ...<.4I.T.abc006
| 3904: 78 79 7a 00 00 00 00 00 00 c3 88 00 c2 ca 4c 4d xyz...........LM
| 3920: d3 23 05 05 06 1f 16 07 59 37 11 10 e9 e5 3d d5 .#......Y7....=.
| 3936: 61 62 63 30 30 35 78 79 7a 00 00 00 00 00 c3 c0 abc005xyz.......
| 3952: 15 12 67 ed 4b 79 22 04 05 06 1f 14 07 93 39 01 ..g.Ky........9.
| 3968: 7f b8 c7 99 58 61 62 63 30 30 34 78 79 7a 00 00 ....Xabc004xyz..
| 3984: 09 c0 43 bf e0 e7 6d 70 fd 61 21 03 05 06 1f 12 ..C...mp.a!.....
| 4000: 07 b6 df 8d 8b 27 08 22 5a 61 62 63 30 30 33 78 .....'..Zabc003x
| 4016: 79 7a 00 00 00 c3 c7 ea 0f dc dd 32 22 20 02 05 yz.........2. ..
| 4032: 06 1f 10 07 2f a6 da 71 df 66 b3 b5 61 62 63 30 ..../..q.f..abc0
| 4048: 30 32 78 79 7a 00 00 c3 ce d9 8d e9 ec 20 45 1f 02xyz........ E.
| 4064: 01 05 06 1f 0e 07 5a 47 53 20 3b 48 8f c0 61 62 ......ZGS ;H..ab
| 4080: 63 30 30 31 78 79 7a 00 c3 c9 e6 81 f8 d9 24 04 c001xyz.......$.
| page 3 offset 8192
| 0: 0a 00 00 00 14 0e fd 00 0f f3 0f e6 0f d9 0f cc ................
| 16: 0f bf 0f b2 0f a5 0f 98 0f 8b 0f 7e 0f 71 0f 64 ...........~.q.d
| 32: 0f 57 0f 4a 0f 3d 0f 30 0f 24 00 00 00 00 00 00 .W.J.=.0.$......
| 3824: 00 00 00 00 00 00 00 00 00 00 00 00 00 0c 03 06 ................
| 3840: 01 7f 46 91 03 3f 97 fb f7 11 0c 03 06 01 6e a2 ..F..?........n.
| 3856: a3 64 68 d4 a6 bd 0b 0c 03 06 01 6d 85 7b ce d0 .dh........m....
| 3872: 32 d2 54 10 0b 03 06 09 5a 47 53 20 3b 48 8f c0 2.T.....ZGS ;H..
| 3888: 0c 03 06 01 59 37 11 10 e9 e5 3d d5 05 0c 03 06 ....Y7....=.....
| 3904: 01 50 f9 4a bb a5 7a 1e ca 0a 0c 03 06 01 48 45 .P.J..z.......HE
| 3920: ab e0 8c 7c ff 0c 0d 0c 03 06 01 36 75 e9 a2 bd ...|.......6u...
| 3936: 05 04 ea 0e 0c 03 06 01 2f a6 da 71 df 66 b3 b5 ......../..q.f..
| 3952: 02 0c 03 06 01 15 f4 c9 23 af e2 b3 b6 14 0c 03 ........#.......
| 3968: 06 01 dd f2 2a a5 7e b2 4d 82 13 0c 03 06 01 d9 ....*.~.M.......
| 3984: ab ec bf 34 51 70 f3 0f 0c 03 06 01 be 6d 1e db ...4Qp.......m..
| 4000: 61 5d 80 9f 0c 0c 03 06 01 b6 df 8d 8b 27 08 22 a]...........'..
| 4016: 5a 03 0c 03 06 01 97 3c bc 34 49 94 54 ab 06 0c Z......<.4I.T...
| 4032: 03 06 01 93 39 01 7f b8 c7 99 58 04 0c 03 06 01 ....9.....X.....
| 4048: 90 8e 1d d9 1c 3a e8 c1 09 0c 03 06 01 8f 8f f5 .....:..........
| 4064: c4 35 b6 7f 8d 12 0c 03 06 01 8b 20 e5 68 11 13 .5......... .h..
| 4080: 55 87 07 0c 03 06 01 86 65 f6 7c 50 7a 2b 06 08 U.......e.|Pz+..
| page 4 offset 12288
| 0: 0a 00 00 00 14 0f 62 00 0f 7a 0f a1 0f c9 0f d9 ......b..z......
| 16: 0f 81 0f d1 0f f1 0f f9 0f e1 0f 89 0e 6a 0f c1 .............j..
| 32: 0f 91 0f 99 0f b9 0f 72 0f 62 0f e9 0f b1 0f a9 .......r.b......
| 3936: 00 00 07 04 01 01 01 11 0e 9e 07 04 01 01 01 0b ................
| 3952: 31 16 07 04 01 01 01 10 37 36 06 04 09 01 01 ab 1.......76......
| 3968: 58 07 04 01 01 01 05 1c 28 07 04 01 01 01 0a 10 X.......(.......
| 3984: cf 07 04 01 01 01 0d b2 e3 07 04 01 01 01 0e d3 ................
| 4000: f2 07 04 01 01 01 02 41 ad 07 04 01 01 01 14 3e .......A.......>
| 4016: 22 07 04 01 01 01 13 27 45 07 04 01 01 01 0f ad .......'E.......
| 4032: dd 07 04 01 01 01 0c 2e a1 07 04 01 01 01 03 df ................
| 4048: e1 07 04 01 01 01 06 59 a7 07 04 01 01 01 04 27 .......Y.......'
| 4064: bd 07 04 01 01 01 09 d0 e0 07 04 01 01 01 12 39 ...............9
| 4080: 4f 07 04 01 01 01 07 c4 11 06 04 00 00 00 00 00 O...............
| end crash-7b75760a4c5f15.db
}]} {}
do_test 5.1 {
set R [sqlite3_recover_init db main test.db2]
catch { $R run }
list [catch { $R finish } msg] $msg
} {0 {}}
finish_test

View File

@ -490,7 +490,7 @@ static sqlite3_stmt *recoverPreparePrintf(
*/
static sqlite3_stmt *recoverReset(sqlite3_recover *p, sqlite3_stmt *pStmt){
int rc = sqlite3_reset(pStmt);
if( rc!=SQLITE_OK && p->errCode==SQLITE_OK ){
if( rc!=SQLITE_OK && rc!=SQLITE_CONSTRAINT && p->errCode==SQLITE_OK ){
recoverDbError(p, sqlite3_db_handle(pStmt));
}
return pStmt;

View File

@ -1,5 +1,5 @@
C Fix\sanother\sproblem\sto\sdo\swith\srecovering\sfrom\sin-memory\sdatabases.
D 2022-10-27T19:06:42.311
C Fix\sanother\scrash\sin\sthe\srecover\sextension\striggered\sby\sa\scorrupt\sdatabase.
D 2022-10-27T20:27:45.594
F .fossil-settings/empty-dirs dbb81e8fc0401ac46a1491ab34a7f2c7c0452f2f06b54ebb845d024ca8283ef1
F .fossil-settings/ignore-glob 35175cdfcf539b2318cb04a9901442804be81cd677d8b889fcc9149c21f239ea
F LICENSE.md df5091916dbb40e6e9686186587125e1b2ff51f022cc334e886c19a0e9982724
@ -385,12 +385,12 @@ F ext/rbu/rbuvacuum4.test a78898e438a44803eb2bc897ba3323373c9f277418e2d6d76e90f2
F ext/rbu/sqlite3rbu.c 8737cabdfbee84bb25a7851ecef8b1312be332761238da9be6ddb10c62ad4291
F ext/rbu/sqlite3rbu.h 1dc88ab7bd32d0f15890ea08d23476c4198d3da3056985403991f8c9cd389812
F ext/rbu/test_rbu.c 03f6f177096a5f822d68d8e4069ad8907fe572c62ff2d19b141f59742821828a
F ext/recover/dbdata.c a7b75b53054d131355cb62fd00643fdafc561dfd1e9e9dd0710778e690579853
F ext/recover/dbdata.c 4c36b75735ebb554bd44b91c8788c45131c6ae1c5e6153eaaf0a189a07eb2448
F ext/recover/recover1.test e08dc7a0513eab9de33e7b8e2260b9538bedb57c9bd6fbb278f328d29a102827
F ext/recover/recover_common.tcl 6679af7dffc858e345053a91c9b0a897595b4a13007aceffafca75304ccb137c
F ext/recover/recoverclobber.test 294dcc894124ab4ca3a7b35766630742a3d25810fceac22220beb64f70a33a60
F ext/recover/recovercorrupt.test 6540aae95e17398dd70b44518367fd56588c44962cb276d2623a0fedba9efe9e
F ext/recover/recovercorrupt2.test c1a703d1612ff7ad8c9c2b86036c195f06ffa5663aedd7f6314074cdb5a56b1f
F ext/recover/recovercorrupt2.test a7e0735cefb79de7959ebd1ee6d963f9505305fe7983ac58394eb5f5aa9236c7
F ext/recover/recoverfault.test 3a0a32b9fc216592b97775d69220695b0926980c0f7424b7a59144e47d7cb568
F ext/recover/recoverfault2.test 321036336af23e778a87f148c4cc4407f88fbdab1fd72ddb661669be9020d36b
F ext/recover/recoverold.test 46e9d99b595fac583d4c67f74d7d89c20a435c752ef6eeb3e918b599940c88e0
@ -398,7 +398,7 @@ F ext/recover/recoverpgsz.test 93e970eab05e4e89f8fd6b1bd23f9ec137ea09857e66ba0d4
F ext/recover/recoverrowid.test 1694a1a5526d825f71279f3d02ab02a1ee4c5265de18858bf54cb8ec54487ac8
F ext/recover/recoverslowidx.test f356bb9fba7ffd6fc50e045e419464f0129ac6e24decf6e919584f79c3493727
F ext/recover/recoversql.test f9872ff2114e13ffd8ee31e1de06919f62b9b48bc080191b5bd076d10becb60f
F ext/recover/sqlite3recover.c b8f4b3a58bc81f2d31ca4645a7dddfc4dedd9a06e66471f827932cc63edc2bc0
F ext/recover/sqlite3recover.c 69656992f1dd3b0645c30e465372bb73c6f64f9620845622424fec8f84a8b42b
F ext/recover/sqlite3recover.h f698ccc94bd4da38761035415ad08c4549a408491ff9fd5f52d34d2214f64e36
F ext/recover/test_recover.c 61ec931e47abca6b2210f46239cafd9f3060741605e3d3c45a7c7a53f63dd957
F ext/repair/README.md 92f5e8aae749a4dae14f02eea8e1bb42d4db2b6ce5e83dbcdd6b1446997e0c15
@ -2052,8 +2052,8 @@ F vsixtest/vsixtest.tcl 6a9a6ab600c25a91a7acc6293828957a386a8a93
F vsixtest/vsixtest.vcxproj.data 2ed517e100c66dc455b492e1a33350c1b20fbcdc
F vsixtest/vsixtest.vcxproj.filters 37e51ffedcdb064aad6ff33b6148725226cd608e
F vsixtest/vsixtest_TemporaryKey.pfx e5b1b036facdb453873e7084e1cae9102ccc67a0
P 347c575108bc8112613a02afda1247bdbed24c15def7eb412d0b27aba047715b
R 8cb4c38216254872472236af72461bb8
P 5a7bfd4a217cd80882a1827674b479cdc547419a785e06e0ee82cb8cfca42701
R 4890ae4a27813f81579cbe6a09f4e6de
U dan
Z 43cd6d4bbed8e35cf002f980c0324c18
Z 5b83e6d937b65a5473d327a12ed454d5
# Remove this line to create a well-formed Fossil manifest.

View File

@ -1 +1 @@
5a7bfd4a217cd80882a1827674b479cdc547419a785e06e0ee82cb8cfca42701
d125377378916fb3147612a536fde15ee955176eea9ea6eaa4a2ee5f1e8e1cbe